:10000000A928A701A901A8000130A50029082702F5
:10001000031D0C2828082602043003180130031998
:1000200002302505031D0130A528A401AA00AB015B
:10003000A01124080319A0150430A3002B0E2520BD
:100040002B0825202A0E25202A080F39F63E0318F2
:10005000073E0A3E4B28A401AA00AB01A0112408C8
:100060000319A0150530A3002730A9001030442043
:100070000330A900E8304420A90164304420A901DC
:100080000A3044202A084B28A8002B08A7002A0879
:10009000A60089202608A600A3030319A01124089E
:1000A00003195528230203185C282608031DA011F4
:1000B000A0195C28303E622808000C1E5D289900BB
:1000C0000314A52821195D28080083178001840ADC
:1000D000FF3E031D6628A528A901A800FF30A80738
:1000E000031CA907031CA5280330A700E7307A20CA
:1000F0006E28A701FC3EA600A709031C8528FF3037
:100100000000A60703188028A6070000A70F7F2875
:100110000800AB01AA011030AC00270DAA0DAB0DF1
:100120002808AA022908031C290FAB0203189F28DC
:100130002808AA0729080318290FAB070310A60DE2
:10014000A70DAC0B8D282608A52883138312031353
:1001500008008316403099002030980083129030B8
:100160009800A00107309F0083168117861406149B
:100170000514851485110511861186128312051147
:100180008511861186122030840060306620A030F0
:1001900084005030662020308400303065204D309F
:1001A0005D2061305D206E305D2020305D20493063
:1001B0005D206E305D2020305D2054305D20683041
:1001C0005D2065305D2020305D204D305D20693040
:1001D0005D2064305D205D206C305D2065305D20E9
:1001E00020305D2062305D2065305D2074305D2000
:1001F00077305D2065305D205D206E305D202030E1
:100200005D2074305D2077305D206F305D202030C0
:100210005D2054305D2049305D2020305D20473026
:100220005D2072305D2061305D2070305D2068306F
:100230005D2069305D206E305D2067305D202030AC
:100240005D2043305D2061305D206C305D20633087
:100250005D2075305D206C305D2061305D20743034
:100260005D206F305D2072305D2073305D200A307C
:100270005D200D305D2028305D2063305D20293009
:100280005D204C305D204A305D2050305D2056307E
:100290005D2020305D2032305D2030305D203130F7
:1002A0005D2030305D20612905158615851586167F
:1002B0000430A900B0306D20051186118511861219
:1002C0000800B201B301AF01030106180130AE000E
:1002D000030105180130AE05030186180130AE0593
:1002E000030185180130AE05031977296429061822
:1002F000972986158515030106180130AE000130D7
:1003000085180301AE0503197B2986118511851C0B
:1003100087293208A200A601A20A0314A60DA20B87
:100320008E292608FF3AB005B20AAF017729861850
:10033000B62986160515030186180130AE00013076
:1003400005180301AE0503199B2986120511051C2A
:10035000A7293208A200A601A20A0314A60DA20B27
:10036000AE292608B004B20AAF0177290518D629AC
:1003700005158616030105180130AE0001308618F8
:100380000301AE050319BA2905118612861CC62978
:100390003308A200A601A20A0314A60DA20BCD29C0
:1003A0002608FF3AB105B30AAF0177298518F52968
:1003B00085158615030185180130AE000130061839
:1003C0000301AE050319DA2985118611061CE629F9
:1003D0003308A200A601A20A0314A60DA20BED2960
:1003E0002608B104B30AAF017729AF0A2F08A60087
:1003F000FE300120AE00083032020130031D003013
:10040000AE04083033020130031D0030AE0403197E
:100410007729FF302F02031C232A54210A305D2044
:100420000D305D2054305D2049305D204D305D2021
:1004300045305D2020305D204F305D2055305D20FF
:1004400054305D20612908303202031D9F2AB41008
:10045000B30803197E2A54210A305D200D305D2037
:1004600046305D204F305D2055305D2054305D209A
:100470003A305D2020305D2062305D2069305D20A3
:1004800074305D205D2065305D206C305D205D2026
:1004900065305D2072305D2020305D2031305D2080
:1004A00020305D203D305D2020305D200430A100F3
:1004B00032082B2020305D2065305D206E305D20BD
:1004C00020305D2062305D2069305D2074305D2019
:1004D0005D2065305D206C305D205D2065305D20E5
:1004E00072305D2020305D2032305D2020305D2074
:1004F0003D305D2020305D2033082B203418992AB0
:100500000A305D200D305D2047305D2052305D2087
:1005100031305D2020305D2073305D2061305D2002
:1005200079305D2073305D203A305D2020305D20D1
:1005300034140430A1003008152020305D2008302C
:100540003302031D1B2B3410B2080319FA2A54215D
:100550000A305D200D305D2046305D204F305D203B
:1005600055305D2054305D203A305D2020305D20D4
:1005700062305D2069305D2074305D205D20653023
:100580005D206C305D205D2065305D2072305D2027
:1005900020305D2031305D2020305D203D305D20F9
:1005A00020305D200430A10032082B2020305D2057
:1005B00065305D206E305D2020305D2062305D2032
:1005C00069305D2074305D205D2065305D206C30C9
:1005D0005D205D2065305D2072305D2020305D2023
:1005E00032305D2020305D203D305D2020305D20A8
:1005F00033082B20B418152B0A305D200D305D20F8
:1006000047305D2052305D2032305D2020305D204B
:1006100073305D2061305D2079305D2073305D2066
:100620003A305D2020305D20B4140430A100310840
:0E063000152020305D20612963001C2B1E2B3D
:02400E00623F0F
:00000001FF
